:100000000C9483000C94A0000C94A0000C94A0000D
:100010000C94A0000C94A0000C94A0000C94A000E0
:100020000C94A0000C94A0000C94A0000C94A000D0
:100030000C94A0000C94A0000C94A0000C94A000C0
:100040000C94AC030C94F1010C94A0000C94A0004F
:100050000C94A0000C94A0000C94A0000C94A000A0
:100060000C94A0000C94A0000C94A0000C94A00090
:100070000C94A0000C94A0000C94A0000C94A00080
:100080000C94A0000C94A0000C94A0000C94A00070
:100090000C94A0000C94A0000C94A0000C94A00060
:1000A0000C94A0000C94A0000C94A0000000000090
:1000B000240027002A0000000000250028002B0053
:1000C00000000000230026002900040404040404A6
:1000D00004040202020202020303030303030102F7
:1000E00004081020408001020408102001020408C6
:1000F00010200000000700020100000304060000B9
:1001000000000000000011241FBECFEFDAE0DEBFC8
:10011000CDBF11E0A0E0B1E0E6E4F9E002C0059057
:100120000D92A830B107D9F71AE0A8E0B1E001C0FC
:100130001D92AC3CB107E1F70E946D030C94A10441
:100140000C9400007F928F929F92AF92BF92CF92B9
:10015000DF92EF92FF920F931F93CF93DF938091E3
:10016000C00A9091C10A01969093C10A8093C00A77
:10017000C39709F4C6C040910301E42EFF24709098
:10018000C20A61E070E0072C02C0660F771F0A9474
:10019000E2F712E0C12ED12C072C02C0CC0CDD1CE2
:1001A0000A94E2F703E010E0072C02C0000F111FD1
:1001B0000A94E2F7B0900501AB2CA09420E030E067
:1001C00049010894811C911CC901880F991F820F55
:1001D000931F9C01220F331F220F331F220F331F47
:1001E000280F391F220F331FE901C85FDE4FC401FA
:1001F000880F991F880D991DFC01EE0FFF1FEE0F50
:10020000FF1FEE0FFF1FE80FF91FEE0FFF1FE85F44
:10021000FE4FD901AC58BE4F51E00DC0822F90E087
:100220000817190799F13A2131835F5F21963196BA
:100230001196553399F12981242388818423280F2D
:100240008A818423280F80818423280F828184233C
:10025000280F8C918423280F11968C911197842359
:10026000280F12968C9112978423280F3181832FA7
:1002700090E08E219F218617970781F6822F90E0CC
:100280008C159D0519F08017910769F63B2931837C
:100290005F5F219631961196553369F68CE2881688
:1002A000910411F094018CCF209104012093C20A93
:1002B000B092030170920401409305018091BD0A40
:1002C0009091BE0A039709F48AC08091BD0A90916B
:1002D000BE0A0597D0F381E090E09093BE0A809328
:1002E000BD0A2093BC0ADF91CF911F910F91FF901F
:1002F000EF90DF90CF90BF90AF909F908F907F90C6
:10030000089581E090E09093C10A8093C00AD09054
:10031000030180E00E943C047C0180E00E943C04D8
:100320006AE270E00E947A04082F0E5F10E0F80184
:100330003197C70162E370E00E947A048E5F90E01B
:100340009F01220F331F2E0F3F1FF901EE0FFF1FDA
:10035000EE0FFF1FEE0FFF1FE20FF31FEE0FFF1F49
:10036000DF01A85FBE4FA80FB91F1196DC92E80FFE
:10037000F91FE85FFE4FD0829801220F331F200F34
:10038000311FF901EE0FFF1FEE0FFF1FEE0FFF1FD2
:10039000E20FF31FEE0FFF1FDF01A80FB91FA85FC9
:1003A000BE4FDC92E80FF91FE95FFE4FD0820F5F6E
:1003B0001F4FF801EE0FFF1FE00FF11F9F01220FEB
:1003C000331F220F331F220F331FE20FF31FEE0FD5
:1003D000FF1FE80FF91FE85FFE4FD082CCCE5E9A78
:1003E00074CF1F920F920FB60F9211241F932F9369
:1003F0003F934F935F936F937F938F939F93AF93AD
:10040000BF93EF93FF9380910001909101010196BA
:10041000909301018093000180910001909101016E
:100420008753914008F092C080918400909185009C
:10043000837090708130910509F43EC1813091053F
:1004400008F039C0000000000000000015B884E08A
:1004500090E00E94F40381E085B989E090E00E9479
:10046000F4038091000190910101849790F08091B4
:100470000001909101018C52914058F44091BF0AC3
:10048000453010F11092BF0A809102018F5F809376
:100490000201FF91EF91BF91AF919F918F917F9159
:1004A0006F915F914F913F912F911F910F900FBED0
:1004B0000F901F9018958230910509F4FAC00397A8
:1004C00029F600000000C2CF8091020190E09C015B
:1004D000220F331F280F391FC901880F991F880F5A
:1004E000991F880F991F820F931F880F991FFC0176
:1004F000E75FFE4F9C01235C3E4F9091BC0A82E077
:1005000085B9913009F4DDC0000091E08191880F38
:10051000816095B985B900000000E217F307B0F3D8
:10052000000000000000000091E095B982E085B96C
:1005300000000000000000000000000000000000BB
:10054000000095B94F5F4093BF0AA3CF15B882E072
:1005500090E00E94F40311E015B98EE190E00E9452
:10056000F40315B882E090E00E94F40315B98EE11F
:1005700090E00E94F40315B882E090E00E94F4033A
:1005800015B98EE190E00E94F40315B882E090E086
:100590000E94F40315B98EE190E00E94F40315B8AF
:1005A00082E090E00E94F40315B98EE190E00E9491
:1005B000F40315B882E090E00E94F40315B98EE1CF
:1005C00090E00E94F40315B88CE190E00E94F403DF
:1005D00015B984E090E00E94F40315B88CE190E036
:1005E0000E94F40315B984E090E00E94F40315B86A
:1005F0008CE190E00E94F40315B984E090E00E9441
:10060000F40315B88CE190E00E94F40315B984E07E
:1006100090E00E94F40315B88CE190E00E94F4038E
:1006200015B984E090E00E94F40315B882E090E0F0
:100630000E94F40315B98EE190E00E94F40315B80E
:1006400082E090E00E94F40315B98EE190E00E94F0
:10065000F40315B882E090E00E94F40315B98EE12E
:1006600090E00E94F40315B882E090E00E94F40349
:1006700015B98EE190E00E94F40315B882E090E095
:100680000E94F40315B98EE190E00E94F40380917A
:10069000BD0A9091BE0A01969093BE0A8093BD0A4E
:1006A00086E090E090930101809300011093020195
:1006B000BBCE00000000CACE000000000000000019
:1006C000C5CE91E081918160000095B985B90000A7
:1006D0000000E217F307B0F325CF0E94020480E880
:1006E000809361001092610088E061E00E945A04EA
:1006F00089E061E00E945A04569A5E9881E08093F6
:10070000C8058093C7058093FD058093FC05809301
:100710003306F89480918100877E88608093810001
:10072000809180008C7F8093800080918100887F01
:1007300081608093810080E094E0909389008093B1
:10074000880080916F00826080936F0010926E002D
:1007500078940E94A200FDCF1F920F920FB60F92C5
:1007600011242F933F938F939F93AF93BF938091C7
:10077000C70A9091C80AA091C90AB091CA0A3091DB
:10078000CB0A0196A11DB11D232F2D5F2D3720F01F
:100790002D570196A11DB11D2093CB0A8093C70A46
:1007A0009093C80AA093C90AB093CA0A8091C30A59
:1007B0009091C40AA091C50AB091C60A0196A11DE4
:1007C000B11D8093C30A9093C40AA093C50AB09345
:1007D000C60ABF91AF919F918F913F912F910F903A
:1007E0000FBE0F901F901895019759F0FC01EE0F66
:1007F000FF1FEE0FFF1F32978FB7F8943197F1F775
:100800008FBF0895789484B5826084BD84B581607B
:1008100084BD85B5826085BD85B5816085BDEEE608
:10082000F0E0808181608083E1E8F0E08081826097
:100830008083808181608083E0E8F0E08081816056
:100840008083E1EBF0E0808184608083E0EBF0E086
:10085000808181608083EAE7F0E08081846080832A
:1008600080818260808380818160808380818068D4
:1008700080831092C10008958F7090910601929527
:10088000990F990F907C982B90937C0080917A001F
:10089000806480937A0080917A0086FDFCCF20915D
:1008A000780040917900942F80E030E0282B392B9C
:1008B000C9010895282F30E0C90182529F4FFC01E1
:1008C000949126533F4FF9018491882391F0E82FAA
:1008D000F0E0EE0FFF1FE455FF4FA591B4916623A2
:1008E00029F48C91909589238C9308958C91892B70
:1008F0008C93089597FB092E07260AD077FD04D024
:100900000CD006D000201AF4709561957F4F0895A1
:10091000F6F7909581959F4F0895AA1BBB1B51E157
:1009200007C0AA1FBB1FA617B70710F0A61BB70B5F
:10093000881F991F5A95A9F780959095BC01CD0104
:060940000895F894FFCFBA
:0809460036010101010201006C
:00000001FF
